:030000000203D721
:03004300020100B7
:1001000002013C000201580002011800020129000E
:10011000020120000201180032E591C2E4F59122AB
:10012000C0E0C2003119D0E032C0E0E5874401F5FB
:10013000870000003119D0E032C2DC32C0D0C0E00C
:10014000C082C08312016931197401907FABF0D075
:1001500083D082D0E0D0D032C0D0C0E0C082C08393
:090160001206833119740280E2D9
:10016900907FE8E0A2E79202545C7051E0A2E0823D
:10017900E1404A30E50274035403C4F540A3E05456
:100189000F45401201D52001343002182003209078
:100199007F027846754003E6F0158218D540F8E6E7
:1001A900907FB5F0754002907FB4E04540F022851C
:1001B9008240E583907FD4F0E540A380E675400353
:1001C90080E5E02582F58250020583229001FA310B
:1001D900CCE09001FA31CCC082C0837845E4F618AE
:1001E900F6187601907FEAE0F5F0A3E0C201C203B8
:1001F900227140404040408A406A78404040404037
:1002090040754040404040B440404040404040403C
:10021900407542404040404040404040404040409E
:1002290040405663404040404040435D404040406C
:1002390040D201223000FA907FC5F0907FAAE054A5
:100249000160FBF002043F3000E708761822300015
:10025900E0F541223000DA08A641223000D508A68F
:10026900462208760122760222E5F0600BC3950347
:1002790050BF85F046D20022C20022D20314900258
:10028900E060B0149002F230F10390033360A414DB
:10029900709F900365E5F0602AF54031CBE06091ED
:1002A900E5401480F2D203C3942190030430F10392
:1002B90090034560C51490031430F10390034E6018
:1002C900B9413AE0FFF5F07800F208A3E0DFFAD08F
:0702D900E0D0E0E5F021A9EF
:1002E0001201010100000040424200010001010230
:1002F000000209022200010103803209040000010A
:1003000003000000092100010001221F00070581F0
:10031000034000640600FF0901A10119012902152B
:100320000026FF00750895288102190129029529E8
:100330009102C009021B000102048032090400007E
:10034000000300000009210001000122170006003F
:10035000FF0901A10119012902150026FF007508F6
:1003600095299102C0040309042C0355005300424F
:10037000002000440065007300690067006E0020E3
:10038000004200790020004500780061006D007097
:10039000006C0065001A035200650061006400658E
:1003A000007200200042006F0061007200640014BF
:1003B00003540065007800740020004D006F006455
:1003C000006500120344006F00740020004D006FB0
:1003D000006400650000007581EB75927F78D6E2BD
:1003E00054F3F212042EE24406F2E4F520F54678C6
:1003F000487F2B7408F608DFFC7893E4F2799CF4CC
:10040000F37895799EE254F0F2E3440FF37898E2A2
:1004100054F0F278ACF208F2087403F2087401F2B6
:1004200078AA74FFF275E80175A8C00080FD7540D8
:100430006490FB50A3E582458370F9D540F3229088
:100440007EC0E0B4020D907EC17849E07F28E0F6DE
:10045000DFFC22758601907EC178497F07E030E796
:1004600002743FC394205002743C75F005A40586C5
:100470009004A32582F582E5F03583F5837E05E0BF
:10048000F6A308DEFA7600080586A3DFD00586907D
:100490007E8078497F28E6F0A308DFFA907FB77462
:1004A00028F022000000000000007D000000700025
:1004B0007000147F147F14122A7F2A2462640813A8
:1004C0002336495522050050600000001C224100DF
:1004D0000041221C0014083E081408083E080800C9
:1004E00005060000080808080800030300000204CD
:1004F0000810203E4549513E00217F01002143451F
:10050000493142415169460C14247F0472515151C2
:100510004E1E2949490640474850603649494936E8
:100520003049494A3C003333000000656600000052
:1005300008142241141414141441221408002040F9
:1005400045483026494F413E3F4848483F7F49494A
:1005500049363E414141227F4141221C7F49494960
:10056000417F484848403E4149492F7F0808087F5D
:1005700000417F41000201417E407F081422417FFB
:10058000010101017F2018207F7F1008047F3E4178
:1005900041413E7F484848303E4145423D7F484CBE
:1005A0004A31314949494640407F40407E0101017E
:1005B0007E7C0201027C7E010E017E6314081463BE
:1005C00070080708704345495161007F4141007F31
:1005D0004141417F0041417F001020402010010136
:1005E0000101010040201000021515150F7F0911AF
:1005F000110E0E111111020E1111097F0E15151594
:100600000C083F484020182525253E7F0810100F74
:1006100000115F01000201115E007F040A11000059
:10062000417F01001F100C100F1F0810100F0E113A
:1006300011110E1F14141408081414141F1F08108D
:1006400010080915151502107E1101021E01010185
:0E0650001F1C0201021C1E0106011E110A04DD
:10065E000A11180505051E1113151911000836414A
:10066E000000007F0000004136080008082A1C0820
:10067E00081C2A0808D54A37754A19789879967A47
:10068E0001E548B4271A907F9CE4F0740CF2799936
:10069E00E3F54779967410F274FFF07A0B7548FF04
:1006AE00E4F3EAF2E4F20548E5482449F8E6F322D9
:00000001FF
